:060000008a016400c8291a
:080008008c00030e8d0020089e
:100010008200cd3081000b116400970ad2280b308a
:1000200001029800903081008b160b110b126400b6
:100030008f150f1d11211e30a000d2288d30810098
:100040000b11023097072630a000d228e330810040
:100050000b11033097072e30a000d2287230810098
:100060000b11040898002308840083160008840af2
:1000700082003a283b283c283d283e283f2840283b
:10008000412842284328442845284628472848280c
:1000900049284a284b284c284d284e284f285028bc
:1000a000512852285328542855285628572858286c
:1000b00059285a285b285c285d285e285f2860281c
:1000c00061286228632864286528662867286828cc
:1000d00069286a286b286c286d286e286f2870287c
:1000e000712872287328742875287628772878282c
:1000f00079280008840a82007d2800088600840a86
:100100000008840a000082008528000886008828ec
:1001100090288a280008860090288e2800088600eb
:10012000f939860096289428000886000b1d962829
:1001300083128b120b110b168b100f30a0008f1136
:1001400002309707a1011808840019088316860059
:100150008312d228cd3081000b116400970a1c0b4a
:10016000be28991519161a080319bd289a1bbb2811
:1001700099119a03bd2819129a0a3c309c001e3c22
:10018000031dce28991799161b080319ce289b1b0f
:10019000cc2899129b03ce2899139b0a1908831621
:1001a000860083120d0e83008c0e0c0e0900640075
:1001b000960197010108a1000518d7288b1efd2084
:1001c00004301702031cdc28043097028001083039
:1001d0000f1c073090008b1efd200d301702031cf2
:1001e000eb280d309702050c800c900beb280310c8
:1001f0000f1c800c051cfa2808006400210801026d
:100200000f158f190f29a1079d009e019d0d9e0db1
:100210001d0d9e0d96071e080318013e97070f112e
:10022000080021081802a10798009c01980d9c0d58
:10023000180d9c0d96071c080318013e970708002f
:100240009d0000079e009d1f2b29801f32299e1ba9
:100250003229803032299d1b3229801b32299e1f72
:1002600032297f309e009e1b3b2940301e021e0813
:1002700003184030402940301e071e08031cc030c0
:100280009e001d081e0208002430950084002308eb
:10029000243c031d4e292a3095008400fd308e0039
:1002a0001a083f3993001b083f39940013020319c1
:1002b0006429031c6629fb308e0013089d00140876
:1002c00093001d0894006629f9308e009d011308e3
:1002d0009402130803197529ff3e03197429ff3e80
:1002e000793c8000840a75299d031408031982292a
:1002f000ff3e03198429ff3e03198629ff3e031997
:1003000088299129943089298e3089298a30892930
:1003100085301d078000840a19080e058000840ab4
:10032000af297d301d078000840a19080e05800062
:10033000840a043014020319a829ff3e0319a629d0
:1003400006301402793c8000840aa829ff30031982
:100350000030943e8000840a1908f939800015089d
:10036000a3000800003092001708031db429920f63
:10037000b42911308400d7207f3000057f3c031959
:10038000bb29f83000050319c62908000f1408001e
:100390008f019a019b01ff309900a50083168c30d4
:1003a0008100831205198f14051d8f1006308600f9
:1003b0002430a3009430a4000930a00081018b16e2
:1003c0008b17b2218b138f18ea293c309c000b113c
:1003d000aa30f3298316f930860083128b120b1191
:1003e0000b168b100f30a0008b170f18fa298f18df
:1003f0005a2a022a8f188c2a342a11308400d720d6
:10040000001fff29801e1917801a1913001e991446
:10041000001a9910840ad720001b552a910c910cc0
:10042000110cc03980041a0820219a07d720001b1c
:10043000552a910c910c110cc03980041b08202105
:100440009b0711308400d720001b022a801e19153b
:10045000801a1911fd2911308400d7207830000549
:10046000031d2d2a801f2d2a00191917001d19138d
:1004700000189914001c991080181915801c191166
:10048000d7201a0820219a07d7208009800a1b0844
:1004900020219b07d7201a0820219a07d7208009fe
:1004a000800a1b0820219b072b2a11308400d720ab
:1004b000001f572a801e1917801a1913001e99173a
:1004c000001a9913840ad720001b552a910c910c0d
:1004d000110cc03900049a07d720001b552a910c33
:1004e000910c110cc0390004ff3a013e9b074421d6
:1004f00011308400d720001b5a2a801e9916801aba
:1005000099124421552a11308400d72078300005f3
:10051000031d852a801f852a00191917001d19132c
:1005200000189917001c991380189916801c9912ad
:10053000d72000089a07d72000089b0744211130d4
:100540008400d72000089a07d72000089b07442181
:02055000832afc
:02400e00fd3f74
:00000001ff
